:100000002FC449C448C447C446C445C444C4C6C632
:1000100042C441C440C43FC43EC43BC660C63BC4A6
:100020003AC439C438C437C4AFC6E3C6E7C6EDC660
:10003000FCC600C70AC71DC735C742C7020408105F
:100040000102020101020100000210040840200226
:100050000201010100000080805F80808080030039
:10006000038080147F147F14242A7F2A122313080C
:100070006462364956205005038080801C224180EE
:100080008041221C808022146B142208083E08083C
:100090005030808080080808088060608080806020
:1000A000100804033E41413E80427F4080806251FF
:1000B00049468022414936801814127F80274545E1
:1000C00039803C4A49318001710D038036494936F7
:1000D000800649291E803636808080563680808092
:1000E0000814224180141414148041221408800240
:1000F00051090680324979413E7E09097E807F4957
:100100004936803E414122807F41413E807F4949BE
:1001100041807F090901803E49493A807F08087F74
:1001200080417F4180802040403F807F0814638071
:100130007F404040807F020C027F7F06187F803E18
:1001400041413E807F090906803E41215E807F0952
:10015000196680264949328001017F01013F4040F4
:100160003F8007186018073F4038403F6314081469
:1001700063030478040361594543807F41418080D3
:10018000030408106041417F8080020102808040AA
:1001900040404080030480808020545478807F4811
:1001A00048308038444428803844447F8038545450
:1001B0004880047E05018048545438807F080870C8
:1001C000807A8080808020403A80807F081462801E
:1001D000417F4080807C047804787C0404788038F7
:1001E000444438807C242418801824247C8078049B
:1001F0000480804854542480043F4444803C404060
:100200007C800C3040308C3C4030403C44281028EE
:10021000444C50503C8064544C44800836418080AB
:100220007F80808080413608808008040810088024
:10023000808080801C2A4949221F047F4040201270
:100240001012201022202210215454798079141485
:100250007980394444398039444439803D40407D77
:10026000803D40403D807E25251A806C1A6F1A6CB7
:100270007D5A1E5A7D4E7B0F7B4E7C3A7E3A7C1C0B
:10028000762E761C1E347C341E0C1224120C081C94
:100290003E7F807F3E1C0880303F01627E303F02FF
:1002A00080801E3D777331607E7B7E60205F23807F
:1002B000807E7A7A7F8003457945031028242810B0
:1002C00008142A1408000000000036360836361ECE
:1002D000143C287844241D244442241D62010865EE
:1002E0001C224146241D244C08443D44084C241D36
:1002F000244601621D620142241D24427C46574669
:100300007C7F2A2A7F802A7F417F2A0A0055000AA3
:1003100030484D33070629792906081C2A080808A1
:10032000082A1C08FE07990770075E070307F306F3
:10033000CF06BA06AF060406A4058A052505FC0407
:10034000AB046E040904D603B70398036F0350038C
:10035000404058646864687048444C48484848487D
:100360004442714952646870705840404040FF1CDC
:10037000222E2A1C1C222A2E1C1C222A2A1C1C2249
:100380002A3A1C1C223A2A1C1C322A2A1C1C2A2A01
:100390002A1C1C262A2A1CFF7F7F7F7F7F1C1C1C97
:1003A0001C1C0808080808080808080800080808AD
:1003B000000000080000FF1C3E773E1C3E7763777C
:1003C0003E7763416377634108416341081C0841FC
:1003D000081C3E1C08FF4040414040404043404014
:1003E00040404540404040494040404051404040EE
:1003F00040214040404051404040484148404840F2
:100400004140484040414040FF00027D0000000163
:100410007C020000007A00000008720400000860FE
:1004200010000010680000002040100000002000B4
:1004300000000000000000000000000000000000BC
:100440000000300000007C543800793D243D797B69
:100450003F163F7B7E7C187C7E7C0810087C7008F1
:1004600010087060082010601040002000FF3F67F7
:1004700064246666246F69693F01003C64662767EF
:10048000663C0000213F69692F29292F69693F21B6
:100490000000203E626223232362623E2000003C73
:1004A000647C243C243C247C643CFF403C433C4032
:1004B000407C437C40403C433C40407C437C40404B
:1004C0003C433C40407C437C40205E215E20106FDA
:1004D000106F100877087708047B047B040275020C
:1004E0007502016801680120502050204010200052
:1004F0004020004000404000400000FF404040409D
:100500004040605048444464544C44446C546C44EF
:10051000446C546C7C446C556E7C446E556E7C7C93
:100520006E556E7CFF40400901000045410000030C
:100530000140400005014040000941400000504199
:1005400001000060410100004051010000004151E4
:100550000000000041490000004141080000404502
:1005600001000005414000030140400105004040FA
:1005700000090140400010014140002041410000BD
:10058000404141000040410100FF20505020003018
:100590004848300006090906000102020100000176
:1005A000010000FF0300000000030000000007003E
:1005B000000000060200000005060000000C060016
:1005C0000000080E0000000A0C040000080A0C00DD
:1005D0000004180C000008101C000000141808008B
:1005E0000010141800000830180000102038000017
:1005F000002830100000202830000000000000001B
:10060000202830FF000007000000000E0000000856
:100610000808001010100000202020000040434374
:100620000000404646000040404C0C00404040184E
:100630001840404060600000002020404040606062
:10064000000107444000020E48400018084C4030AA
:1006500010184040602030404060273440407E30D9
:100660003040407E313340407E323640407E30362E
:1006700044407E30304C487E303050587E303060C0
:10068000705E101040507E303060707C20204060E2
:100690007C212744607C222E48607C38284C607C7A
:1006A0003B2B4C607C3E2E4C607C3F2F4D60FF55B9
:1006B0002A552A552A552A552AFF101010101008BD
:1006C00010100F7010100808101010101010FF00FC
:1006D00026202600002620260000262026000026B0
:1006E0002024000026202600002620260010262098
:1006F0002610FF00001C0000003E223E007F41410A
:10070000417FFF0100000000020001000004000220
:10071000000008010400011002080002200411007A
:1007200004410822000842104401104520480220DC
:100730004A4050044154406008426841601144708E
:100740004260224870446045507048604A50705082
:1007500060546070606068607060607060FF084442
:10076000281008040204085030100804040201FF95
:100770000100000000020201000006090906000055
:1007800030484830002050502000304848300000A9
:100790000609090000000102FF785C6878717C3866
:1007A000747C7A78506262787C606170687A6030BC
:1007B00078747079705269607C6870615066707886
:1007C0002068716072507479706268727030617400
:1007D000617850707A7431406844106870346028D1
:1007E0004A605860607038661860707842195864C2
:1007F000702970703A7854707051786A70FF142ABA
:1008000049493E001C2A493E003E493E087F2A1CB9
:100810000808221C0808081C000808080008080826
:100820000808080808000808080000080800000078
:100830000800000000000000000C0000000C120086
:10084000000C1224000C1224120C1224120CFF3281
:100850001E120B070503020001020305080D150017
:1008600011241FBECFE5D1E0DEBFCDBF10E0A0E672
:10087000B0E0EAEAFFE002C005900D92A836B107A9
:10088000D9F711E0A8E6B0E001C01D92A933B10785
:10089000E1F747D388C3B4CBCF93DF93CDB7DEB7AF
:1008A000C350CDBF809134018F5F80933401853078
:1008B00010F01092340120913401E0913301F0E006
:1008C000E559FF4FE20FF11D308119821A821B8218
:1008D00080E090E030FF11C0FC01ED5BFF4F4491E0
:1008E000FC01E45CFF4FE491A1E0B0E0AC0FBD1F60
:1008F000A40FB11D4C914E2B4C9336950196873029
:10090000910541F780E090E0281789F0FC01E15B58
:10091000FF4F3491FC01E65BFF4FE491A1E0B0E0B2
:10092000AC0FBD1FA30FB11D3C913E2B3C93019614
:100930008530910549F78BB38C7F9981892B8BBBCF
:1009400088B381789A81892B88BB82B3817E9B8111
:10095000892B82BBCD5FCDBFDF91CF910895F09100
:1009600035018F2F8F704F2F50E0BA01607170707A
:10097000E0913301F4FF02C0E81B01C0E80FA09131
:1009800036018E2F90E004962A2F30E082179307CD
:10099000F4F080913801882321F081508093380150
:1009A00014C0809137018093380145FF05C080E174
:1009B0008F278093350109C06115710521F0A5507D
:1009C000A093330102C01092330181E00895E093B7
:1009D000330180E008958F706370613019F04093A7
:1009E000380102C0109238016295682B609335017E
:1009F00040933701089510923301109236011092FE
:100A00006B0010926C0010926D0010926E001092AC
:100A10006F000895F0DF10923501109237010895AC
:100A2000209136010BC0FC0134913F3F49F0019603
:100A3000E22FF0E0E559FF4F30832F5F283C98F319
:100A400020933601089590913601983C40F4E92FA7
:100A5000F0E0E559FF4F80839F5F90933601089542
:100A60008F3D49F0843C61F0863D79F08C3D79F012
:100A7000843E79F002C08AE811C0863F61F002C06E
:100A800085E80CC08C3F49F009C087E807C089E8B9
:100A900005C084E803C086E801C088E88052813937
:100AA00010F5E82FF0E0CF01880F991F880F991FEC
:100AB000EC5AFF4FE80FF91F8091360195E001C015
:100AC000F9019F012F5F3F4FE491E7FD0AC0883C89
:100AD00030F4A82FB0E0A559BF4FEC938F5F915031
:100AE00079F780933601089583E08ABB8EE787BB50
:100AF0008EE181BB8BB38C6F8BBB88B3816888BB65
:100B000082B3816E82BB10BE85E083BF84E086BF66
:100B100087E28CBF89B7856089BF87E689B912B83B
:100B200080E98AB986E083B90895CF93C82F83FFFF
:100B300002C085E001C081E06C2F661F6627661F3A
:100B4000660FEC2FE295E770F0E0E95AF74F449119
:100B500042DFC770EC2FF0E0E15BF74FE491E093E8
:100B60006500CF910895EF92FF920F931F93CF935B
:100B7000DF930F92CDB7DEB77C01FFD1D6DF3BDF2D
:100B800087010E5F1F4FC7010196F7D1982F42C012
:100B900078019E37A1F40894E11CF11CC801EDD145
:100BA0008E3761F1E82FE154E63140F5F0E0EE0FC9
:100BB000FF1FEC5DFC4F8591949132DF1FC09F3F7A
:100BC00081F40894E11CF11CC801D7D107C03BDFB8
:100BD00087010F5F1F4FC701D0D178018F3FB9F751
:100BE0000DC09E3549F40894E11CF11CC801C5D123
:100BF000982F8E3509F0915C892F32DF87010F5FC6
:100C00001F4FC701BAD1982F882321F080E0998324
:100C10001ADF9981992309F0BBCFC801AED188238F
:100C200011F400E010E0C8010F90DF91CF911F9107
:100C30000F91FF90EF900895DEDE8FEF94E3ACE02C
:100C400081509040A040E1F700C0000080E18ABFE1
:100C500090E495B98BBF85B7806585BF85B7806205
:100C600085BF889585B78F7D85BF1BBE83E8F8DE7D
:100C70008FE79AE1A6E081509040A040E1F700C0E4
:100C8000000080E090E06FDF90936300809362004B
:100C900008951F920F920FB60F9211242F933F9336
:100CA0004F935F936F937F938F939F93AF93BF9374
:100CB000EF93FF9386B78C5F86BFEEDDFF91EF91D8
:100CC000BF91AF919F918F917F916F915F914F9164
:100CD0003F912F910F900FBE0F901F9018951F926C
:100CE0000F920FB60F9211242F933F934F935F9360
:100CF0006F937F938F939F93AF93BF93EF93FF93E4
:100D00008CB7895D8CBF80916600882321F081506B
:100D10008093660005C080916500809366001FDEA9
:100D200080B386FF08C08091640080FF1CC0809162
:100D300064008E7712C08091640080FD05C081E060
:100D40008093640084E60DC080916400813059F482
:100D500080916800882321F483E08093640003C0BD
:100D6000815080936800FF91EF91BF91AF919F9167
:100D70008F917F916F915F914F913F912F910F9044
:100D80000FBE0F901F9018951F920F920FB60F92E3
:100D900011240F900FBE0F901F9018951F920F9265
:100DA0000FB60F9211242F933F934F935F936F933E
:100DB0007F938F939F93AF93BF93CF93EF93FF93C3
:100DC0005C999DC0CCB1CB3119F482E0809369006D
:100DD00080916900853018F00EDE8C2F41DEE091A5
:100DE0006900F0E0E930F10508F089C0EB5EFF4FE3
:100DF0000994C83409F083C081E077C0CC3409F489
:100E000073C0C43479F483E070C080E090E09093C4
:100E10006300809362009093610080936000EBDD3B
:100E200081E81EDE109269006AC0E5DD8C2F7DDE50
:100E300084E05BC0CD3011F0CA3011F4DCDD5FC05E
:100E40008C2F0EDE80E0FFDD5AC0CD3011F0CA30AD
:100E500081F480916000909161009C012F5F3F4F71
:100E6000309361002093600060E08FD086E0809333
:100E70006900CE3511F487E038C0C43221F41092F5
:100E80006A0088E032C0C032D0F180916000909159
:100E900061009C012F5F3F4F309361002093600001
:100EA0006C2F21C080916000909161009C012F5FA8
:100EB0003F4F30936100209360006C2F615C13C042
:100EC000C13408F0C750C053C03190F08091600029
:100ED000909161009C012F5F3F4F30936100209300
:100EE000600060916A0051D085E08093690007C07E
:100EF00080916A008295807F8C0F80936A00FF91B9
:100F0000EF91CF91BF91AF919F918F917F916F9111
:100F10005F914F913F912F910F900FBE0F901F90B7
:100F20001895E2DD77DD789487DE80916400806833
:100F30008093640080916400882371F48091620042
:100F40009091630010DE9093630080936200809123
:100F5000640080688093640080916400833051F75E
:100F60004ADD82E87DDD8FE79AE1A6E0815090407E
:100F7000A040E1F700C00000D7CFE199FECF1FBA33
:100F80008EBBE09A99278DB30895262FE199FECF65
:100F90001CBA1FBA8EBB2DBB0FB6F894E29AE19A29
:0A0FA0000FBE01960895F894FFCFEC
:080FAA000000000080080100B6
:00000001FF
